:020000020000FC
:0200000006C038
:10000C006BC04FED4DBF40E0642E4FEF41BB4CEF4A
:10001C0047BB4CE348BB40E048B94FEFA42E7724D4
:10002C0088249924BB2443E043BF40E042BF42E014
:10003C0049BF4FEF642E78944EEA482511F4AA2458
:10004C00A09448EE482579F4F89444274EBD43BF5C
:10005C0048E141BD40E141BD4798442747BB41BB06
:10006C0040E345BF8895BB2029F442E0482511F4B4
:10007C004AE5B42EE1CF20E1FF24EE24DD24FF2756
:10008C00000F111FDD1CEE1CFF1C2A9509F40895AE
:10009C00E0E132913D5F33FD30833081305D37FDDF
:1000AC003083ED30B1F7ECCFF1E0EEECE50F40E052
:1000BC00F41FC895E62FF0E000820895AA2059F0AD
:1000CC0000E013E00A950030E9F71A951030D1F7EB
:1000DC00C298C398C49808954F93AF93BF9340911F
:1000EC005F004F930F931F9341E0740E4427841EBF
:1000FC00941E73957370C298C398C498703039F07D
:10010C00713049F0723059F0733069F051C012BA45
:10011C00C49AD4DF4DC022BAC39AD0DF49C032BAD8
:10012C00C29ACCDF45C061FE43C083958830E1F7AD
:10013C008827C098B89A00E018E00A950030E9F7D3
:10014C00B898B0E0A0E0119748B1459BFCCF4AE5C8
:10015C004B2529F44A2E5B2E4FEFB42EAA24A4195A
:10016C00B50912F4B0E0A0E04B2F4F704350BAF435
:10017C0019F44A2F475E9AF40A2F1B2F7CDF5D2D52
:10018C005F7061E091DF5D2D5695569556955695AD
:10019C0062E08ADF5E2D5F7063E086DF09C05AE0A3
:1001AC0061E082DF5AE062E07FDF5AE063E07CDFEF
:1001BC001F910F914F9140935F00BF91AF914F9161
:0E01CC0018953F065B4F666D7D077F6F090833
:00000001FF
:1001E0008AD120E28FD1089520E28CD120E28AD1F9
:1001F0003E2F81D120E286D108955BE029C1D0E075
:10020000CFEFFF24EE247727BF7D0881CA95E394C2
:100210000D3041F0E1D0523039F0B0625130A9F3E5
:10022000F394F3CF0F2D0895B5FF7395EECF54E0FF
:100230000FC152E00DC19F708F707F70CFD10895B4
:10024000D0E0CFEFE030A9F3088100833197219708
:100250000D30C1F75E2E6F2E0895D1DF743068F631
:10026000062D033021F4052D033F09F452C0D0E0E0
:10027000CFEF772788279927C715CAF20881ACD016
:10028000523029F4982F872F702F2197F5CFD3DF85
:10029000A72EF62DE52DB77FBF7E992788277727D4
:1002A000BB243196F33011F4E43F59F0008194D02F
:1002B000543039F0523089F7B394782F892F902F2A
:1002C000F0CF0B2D033029F0B394782F892F90E0D5
:1002D000F8CFB4FD02C0B061E0CFADDFA71691F159
:1002E00018F4B860DF2ECE2EF33021F4E43F11F481
:1002F000B3FF0FC0B3FF08C07A1508F442C0F33053
:1003000019F4E43F09F43DC0F33039F6E43F29F62F
:10031000089575DF003009F40895D0E0CFEFF62D91
:10032000E52DF23019F4E03009F409C008810083AA
:10033000319721970D30A9F75E2E6F2E089502E0B8
:10034000502F86C03197DF2FCE2FD23019F4C03016
:1003500009F46DCF088121970D30B9F70E2F0C1BD2
:10036000500E08F46394D23011F4C03029F00881A3
:10037000008321973197F7CF42DF003009F06DCF2E
:1003800008953DDF003039F1062D023021F4052DAE
:1003900000500E15A0F2F62DE52DDF2FCE2FCE1931
:1003A000D0400C2F502E0D2F602EFD1519F4EC159A
:1003B00009F405C00081088321963196F6CFD0E07C
:1003C000CFEFFD2DEC2D3197088100830D3019F012
:1003D00031972197F9CF08955527102F1D3009F433
:1003E00016C01F75103009F402C01C3011F451E022
:1003F000089510310AF408951B350AF00895103459
:1004000012F053E008951A310AF452E0089554E0CE
:100410000895CF3F19F427E075D00AC0212F81D06D
:10042000C3951DE0188304C02EE36CD0D0E0CFEF5D
:100430007DD0183071F318831D3049F0C23C19F497
:1004400027E060D0F5CFCA95212F6BD0F1CF08956A
:1004500063D0503021F4F6E0E0EF6CD042C0513070
:1004600021F4F7E0E8E166D03CC0523021F4F7E037
:10047000E6E560D036C0533021F4F7E0E8E75AD023
:1004800030C0543021F4F7E0EAEB54D02AC05530A4
:1004900021F4F7E0ECEE4ED024C0563021F4F8E021
:1004A000E0E248D01EC0573021F4F8E0E2E642D046
:1004B00018C0583021F4F8E0E2EC3CD012C05930BA
:1004C00021F4F9E0E2E236D00CC05A3021F4F9E030
:1004D000EAE530D006C05B3021F4F9E0E2E92AD049
:1004E00000C00FE504E00EBF0FE50DBF6FEFA0E009
:1004F000B0E012D0C3CD57D0242F04D0232F02D088
:100500000895202F5D9BFECF06D6B6FF03C05F9BEC
:10051000FECFBF7B2CB908952DE0F4DF2AE0F2DF97
:1005200008952D3011F4F8DF0895ECCF5F9BFECFD6
:100530001CB10895C895002021F0202DE3DF3196ED
:10054000F9CF0895F7DFE8DF089530DE07E00717F9
:100550004AF001E0703019F0000F7A95FBCF702F50
:100560001CDE08955AE074DF903039F0905D292F39
:10057000C9DF803011F420E3C5DF803019F0805DE1
:10058000282FC0DF705D272FBDDF089599278827AA
:10059000745610F09395FCCF7C597A5010F08395E7
:1005A000FCCF765F0895432F469546954695469530
:1005B000405D4A3308F0495F3F70305D3A3308F0E0
:1005C000395F089546FD475F4F7036FD375F3F70D6
:1005D000440F440F440F440F342B08959330B2F46A
:1005E000923032F0863092F4853012F0763072F428
:1005F000882321F00AE0700F8A9581F7992309F486
:10060000089504E68894700F9A95C0F751E020CFC2
:1006100083DF82DFF6E0ECE195DF089520202020E3
:1006200020204154544F4241534943207665727310
:10063000696F6E203136332D303231313135432EF2
:10064000204E6F7420666F7220636F6D6D657263EC
:1006500069616C207573652E0A0D202020202020F2
:10066000436F70797269676874203230303220626B
:100670007920526963686172642043617070656CAF
:100680007320616C6C207269676874732072657383
:1006900065727665642E0A0D202020202020687463
:1006A00074703A2F2F70726F6A656374732E636172
:1006B0007070656C732E6F726720202020202020C0
:1006C00070726F6A656374734063617070656C7398
:1006D0002E6F72670A0D00004672656520207061FA
:1006E0006765733A0000202063686172733A000006
:1006F0004572726F7220303A20556E6B6E6F776E56
:1007000020636F6D6D616E64206F72206F70657213
:1007100061746F722E2000004572726F7220313A40
:1007200020456E636F756E74657265642061207616
:10073000616C75652074686174206973206E6F74D4
:10074000206265747765656E203020616E642032AA
:1007500035352E2000004572726F7220323A2050DB
:10076000726F6772616D206D656D6F72792069734C
:100770002066756C6C2E00004572726F7220333AE1
:1007800020456E636F756E746572656420612063C9
:100790006861726163746572207468617420697342
:1007A000206E6F742061207265636F676E697A6571
:1007B0006420747970652E2000004572726F72207B
:1007C000343A28696E7465726E616C206572726F5E
:1007D00072202D627566666572206C696D69742081
:1007E0006578636565646564292000004572726FF1
:1007F0007220353A20496E617070726F7072696153
:100800007465207661726961626C65206E616D65E8
:1008100020656E636F756E74657265642E200000CE
:100820004572726F7220363A20446174612073748D
:1008300061636B2070757368206572726F72202D12
:10084000746F6F206D616E7920617267756D656E72
:100850007473206F6E206F6E65206C696E652E203C
:1008600000004572726F7220373A20446174612033
:10087000737461636B20706F70206572726F722E7B
:100880000A0D20202020202020202046756E637431
:10089000696F6E20747269656420746F207573656A
:1008A00020612076616C75652074686174207761C1
:1008B00073206E6F7420617661696C61626C652E65
:1008C00000004572726F7220383A204D616368698A
:1008D0006E6520737461636B206572726F720A0DAE
:1008E00020202020202020202046756E6374696F10
:1008F0006E7320616E642F6F722063616C6C732065
:100900006E657374656420746F6F20646565706CC8
:1009100079206F7220746F6F20636F6D706C6578D3
:1009200000004572726F7220393A20474F544F20B1
:100930006F7220474F5355422064657374696E612E
:1009400074696F6E206C696E6520776173206E6FBD
:100950007420666F756E642E00004572726F72208F
:10096000413A205370656369666965642062697401
:1009700020706F736974696F6E2072616E67652095
:100980006F6620302E2E3720657863656564656458
:1009900000004572726F7220423A204C696E6520E9
:1009A0006E756D62657220686173206D6F7265206F
:1009B0007468616E207468726565206E756D65720D
:1009C000616C732000004C495320C20553495A20E2
:1009D000CE054E455720450850500B203506505047
:1009E0000D203C065052494EE20550525820E90570
:1009F000505242201B0750574D386B065057452028
:100A0000750650574F208106454D49540E07501A20
:100A10001D20F10550501D20FA05464F5220980622
:100A20004E4558540B06501C1E20140650501E20D4
:100A3000840650501C206506504946208E065054AE
:100A40004F209A06505004209E0652554E200C0806
:100A5000454E44209C06414E442043064C535220B0
:100A60004A064C534C204F06504F52205406584FC4
:100A700052205B0644554D505808474F544FD006FE
:100A8000474F5355D40652455455D7065448454E02
:100A900094064B455920130741434F2020065341EC
:100AA0005645DD064C4F4144F6065045454B26065B
:100AB000504F4B452D064F444120DB074F44422009
:100AC000DF074F444320E3074F444420E7074F50DC
:100AD0004120CB074F504220CF074F504320D30730
:100AE0004F504420D707494E4120EB07494E422042
:100AF000EE07494E4320F207494E4420F507534282
:100B000041202707434241202E0753424220360707
:100B1000434242203D07534243204507434243207E
:100B20004C07534244205407434244205B0753443C
:100B300041206307434441206A075344422072071F
:100B400043444220790753444320810743444320D0
:100B50008807534444209007434444209707494260
:100B600041209F0749424220AA0749424320B50736
:100B700049424420C00741444320F90744454C41C1
:100B800076080000C9DCF3E0E3EFF61511F4E51593
:100B900021F02081C6DC3197F8CFBEDCBDDCF6E069
:100BA000E8EDC8DC752D962D70509240F6DA792F5D
:100BB000EDDCDADCF6E0E6EEBDDCF8DAE7DCD4DC2E
:100BC000ABDC0895AE7FB9DAF1DAE0DCCDDCA4DC91
:100BD0000895B2DA24E296DCE9DA372F8CDC9CDC6B
:100BE0000895AE7FAADAE2DA072FE0DAF0E0E72F25
:100BF00000830895A2FF40C0AE7F9FDAD7DAA72E08
:100C0000D5DA872FD3DAB72EF0E0E72F8083A06202
:100C1000A860AA7F0895F0E0EB2D00810A1519F075
:100C200003950083A061089587DAC0DA072FBEDA42
:100C3000701719F07727B1DA08957FEFAEDA0895CB
:100C40007BDA70E0459B71E0A8DA089575DAAEDAD8
:100C5000E72FF0E07081A1DA08956EDAA7DA072FA6
:100C6000A5DAF0E0E02F7083089566DA9FDA072FA7
:100C70009DDA700F92DA08955FDA98DA072F96DA24
:100C8000701B8BDA089558DA91DA072F8FDA702308
:100C900084DA089551DA8ADA76957FDA08954CDAA3
:100CA00085DA770F7ADA089547DA80DA072F7EDA65
:100CB000702B73DA089540DA79DA072F77DA702724
:100CC0006CDA089571E069DA089536DA6FDA072F81
:100CD0006DDA70171EC030DA01E80FBD0EBD8D9AB7
:100CE00065DA00E00BBD7ABD089526DA03E80FBD92
:100CF00001E00EBDBD9A5ADA072F58DA7BBD0ABD56
:100D0000089500E00FBD089517DA50DA072F4EDA84
:100D1000071770E0BAF6B1F240DA08950DDA46DA54
:100D2000772309F0A26008950DB70E5F0DBF0895F7
:100D3000A460089501DA0895B26008954881E5D964
:100D4000388140DC732F29DAE0D9F6D90895F4D937
:100D50002DDA472FF3E0E3EF0AC0F61511F45E1623
:100D6000E8F400810D3011F03197F7CF31977727F4
:100D700088279927F61511F45E1680F400812CDB84
:100D8000523029F4982F872F702F3197F3CF9F700F
:100D90008F707F7023DC471701F7089559E058CB17
:100DA000D6DFDF2FCE2F0895D2DFA06C0895B2FFDB
:100DB00002C0B1600895B26008956FEF752DEDD94E
:100DC000762DEBD9D3E0CFEFEFEFF1E00881E19999
:100DD000FECFFFBBEEBB0DBBE29AE19AD23011F41D
:100DE000C03019F031972197F1CF0895D3E0CFEFBC
:100DF000EFEFF1E0E199FECFFFBBEEBBE09A0DB360
:100E00000883D23011F4C03019F031972197F2CF16
:100E10006DEFCCD9672ECAD9572E08958DD9C6D972
:100E2000272F70DB0895579BFECF7CB1733009F4F8
:100E3000B260B3D9089580D9B9D908E020E3771F0B
:100E400008F421E35FDB0A95C9F766DB089574D9DE
:100E50007CDBACD90BB3072B02BB08956DD975DBD6
:100E6000A5D970950BB3072302BB089565D96DDB37
:100E70009DD908B3072B02BB08955ED966DB96D9CE
:100E8000709508B3072302BB089556D95EDB8ED94F
:100E900005B3072B02BB08954FD957DB87D970954F
:100EA00005B3072302BB089547D94FDB7FD902B3AF
:100EB000072B02BB089540D948DB78D9709502B35F
:100EC000072302BB089538D940DB70D90AB3072B3A
:100ED0000ABB089531D939DB69D970950AB3072364
:100EE0000ABB089529D931DB61D907B3072B07BBAA
:100EF000089522D92ADB5AD9709507B3072307BB77
:100F000008951AD922DB52D904B3072B04BB0895E4
:100F100013D91BDB4BD9709504B3072304BB089589
:100F20000BD913DB43D901B3072B01BB089504D9B7
:100F30000CDB3CD9709501B307230ABB0895FCD89C
:100F400004DB34D909B3072370E0002309F471E00E
:100F500024D90895F1D8F9DA29D906B3072370E026
:100F6000002309F471E019D90895E6D8EEDA1ED904
:100F700003B3072370E0002309F471E00ED908954C
:100F8000DBD8E3DA13D900B3072370E0002309F4B8
:100F900071E003D90895D0D809D97BBB0895CCD886
:100FA00005D978BB0895C8D801D975BB0895C4D8B0
:100FB000FDD872BB0895C0D8F9D87ABB0895BCD8C3
:100FC000F5D877BB0895B8D8F1D874BB0895B4D8D4
:100FD000EDD871BB089579B3E0D8089576B37C7FDE
:100FE000DCD8089573B3D9D8089570B37C7FD5D871
:100FF000089570E0D2D8A0D8D9D87F71706E77B933
:1010000006ED06B93699FECF75B1C7D8089542727C
:1010100065616B200A0D0000D3E0C3EF6FEFA160A4
:101020007AD0A5FF03C0CC2EDD2EAF7DA4FF03C078
:10103000DD2DCC2DAF7EA6FF03C0EC2EFD2EAF7BA9
:10104000A7FF04C0DF2FCE2FB460AF77B0FF03C07F
:10105000DF2DCE2DBA7FB1FF04C043D0D62DC52DD4
:10106000BD7FD61511F45C1678F40881B5D9A1FFBF
:1010700004C0543011F02197D1CFAD7F523011F41C
:101080002197CCCF5AD8CACF0895C2DA03E0602E98
:1010900003EF502EF62DE52D6FEFA0E0B0E000E05D
:1010A000F23011F4E03019F000833197F9CF089550
:1010B000F3E0E3EFF23011F4E03041F030811BDA7D
:1010C00020E220DA20E21EDA3197F4CF25DA24DAA2
:1010D000362D11DA20E216DA352D0DDA1DDA1CDA9A
:1010E0000895F0E1EEE026DA0895189525D85ED847
:1010F0009927882755270027772361F09A958A95A5
:101100005A954A95F1F70A95E1F7D1F7C1F7B1F78A
:101110007A95F2CF0895579B09C00CB1033111F4B1
:10112000B06404C00CB1033009F4B26008950F93A9
:101130000FB72F930F93B395BBBB0F910FBF2F9199
:101140000FBF0F911895002709BF08E002BD0027C7
:1011500004BD03BD05E005BD02B50770E9F708B79A
:0C1160000F7308BF09B7006409BF0895B1
:00000001FF
